:020000020000FC
:10000000A4CDAFC10000000020C0000094C00000DB
:1000100000009EC000000000000000000203040673
:10002000080C10182030406080000406080C1018DE
:100030002030406080A0C00000070F1F3F000D0D62
:1000400004050D050305030302004FB662FD0EC053
:10005000552009F00994C52DC095089483FDC795D6
:10006000C4BDC093A10064604FBE1895C0916400E8
:10007000089483FDC795C4BDC093A1006B7FC09158
:100080006400CF3F09F420C070FF02C082FD05C0AC
:100090004FBE9598AC98C098189575FD0EC065FD3B
:1000A0000CC0C091B300C0FD9498C1FDAD98C2FDD5
:1000B000AB98CAEFC095CA95F1F79598AC98C098DF
:1000C0002092A1004FBE189524BCCC27C064C8BFA5
:1000D0006460F6CFC0CF70FFBECF65FDBCCF959AF0
:1000E000BACF70FFB8CF65FDB6CFAC9AB4CF70FF72
:1000F000B2CF65FDB0CFC09AAECF949A70FFABCFB0
:1001000065FDA9CFC7E0CA95F1F7959AA4CFAD9A3E
:1001100070FFA1CF65FD9FCFC7E0CA95F1F7AC9AFC
:100120009ACFAB9A70FF97CF65FD95CFC7E0CA9580
:10013000F1F7C09A90CF4FB6C9B7CF7EC9BF6E7FD7
:10014000CCB5CE0DDDB5DF1DDBBDCABD4FBE1895EC
:100150003FB68F7EABB7A074A2118061A0E0ABBFA9
:10016000A9B7AE7FA9BF7894A0916800AA2341F0F7
:1001700085FD2AC0A0916800AA95A093680024C0BC
:1001800040E050E085FD14C0A0B396FDA095A2FD0F
:100190004FEFA3E096FDA2E0A5BFAA27A064AABFE7
:1001A0008D7FA0B396FDA095A2FD5FEF451741F7A7
:1001B000A8E161FDA093680085FD03C0A8E1A093BC
:1001C000680040939700816085FD0EC0A091690092
:1001D000AA2331F0A0916900AA95A093690004C0F8
:1001E0008061AA27A064AABF80FF37C0A0919700B2
:1001F0004A2F61FF8E7F85FD1CC0A091B600A43000
:10020000C1F4403F08F040EFA42FA295AF704A0F11
:100210005091B800533069F0A695A69550FD01C0E5
:10022000A69552FD03C0A41B4A2F03C04A0F08F431
:100230004FEF40936100A72FA67079F0A0916D0059
:10024000A695A69556E0A50F50916100A50FA09325
:10025000610018F4AFEFA09361004091B600443004
:1002600009F03EC0A0916100A0936300409163003B
:10027000A0919C004A1708F04A2FA0919E004A17AF
:1002800008F04A2F542EA091A200AA2309F422C0FC
:10029000542F5A1B10F4A42F50E0BA2E8894AA1F92
:1002A000AA2EA091A400A095AA22A50E58F0A09174
:1002B000A300A21509F0AA95AA0EA093A30048F0E6
:1002C0004A2D08C0A091A300BA1608F0A395A093E8
:1002D000A3004FEF409364007F7D485F08F0706299
:1002E000A52DA03408F06860A0916000A395A093AC
:1002F000600051F0F894A9B7A160A9BF84FF02C0C3
:10030000A0E4ABBF3FBE1895A0917400A395A09345
:10031000740041E050916800552329F085FF03C027
:100320005A9550936800A0919700A13018F0209240
:100330009A000DC020929B002092A500A0919A00E7
:10034000AF5FA0939A0018F0AFEFA0939A00F894D3
:10035000A9B7A160A9BF84FF02C0A0E4ABBF3FBEA4
:1003600018953FB64CB55DB58F7EABB7A074A211A2
:100370008061A0E0ABBFA9B7AE7FA9BF789481FD33
:1003800023C0A2E096FDA3E0A5BF8260A0B396FDC6
:10039000A095A2FF05C040936500509366003EC142
:1003A000A3E096FDA2E0A5BFAA27A064AABF8D7F07
:1003B00085FF01C026C140E0A0B396FDA095A2FD37
:1003C00020C1409397000FC1A3E096FDA2E0A5BF16
:1003D0008D7F61FF71C0A2E096FDA3E0A5BFAA27B3
:1003E000A064AABF82604093920050939300A090B3
:1003F00090004A19B09091005B09BB24A22C4C38A4
:10040000520518F42092960049C0A091D600AA2364
:1004100059F1483C520528F4A0E1BA2EAAE0AA2ED0
:1004200023C04836A1E05A0728F4A8E0BA2EAFE06E
:10043000AA2E1AC0403DA2E05A0728F4A4E0BA2E22
:10044000AEE1AA2E11C0403AA5E05A0728F4A2E076
:10045000BA2EACE3AA2E08C04839A8E05A0720F407
:10046000A1E0BA2EA8E7AA2EC42EA0919400CA1A21
:10047000D52EA0919500DA0ADD202AF4AFEFC094C2
:10048000D094CA1ADA0A20929600A8E0A210A0E03E
:10049000CA14DA0618F4A1E0A093960040939400E1
:1004A000509395004091920050919300409390009A
:1004B0005093910002E097C0A09165004A1BA09163
:1004C00066005A0B94FD82C093FD80C092FD7CC0F3
:1004D00086FF03C0D52EC42E0CC05695479591FDBE
:1004E00073C05695479590FD6FC0D52EC42ED694F7
:1004F000C79461FD19C0AC2DAC51AD2DA24008F0E0
:1005000005C0DD2089F4AC2DA85C70F4A0916700D3
:10051000A395AA2311F0A0936700AA3008F471C034
:100520002092970081606DC0A0916700AA2319F006
:10053000AA95A0936700A22C5091BC0097FD06C01D
:10054000A090CA00533011F4A090D200AAEFAA0ED6
:10055000A22DA21DCA18DA0A4FB74170533049F4D0
:10056000442321F087FD05C0806803C087FF01C0D8
:100570008F77442359F0533031F4AFEFC094D094C7
:10058000CA1ADA0A03C040E050E020C0533049F4F0
:10059000CC0CDD1CAAE0CA1AD20818F4A0E0CA2EBE
:1005A000D22CAFEFCA16D20418F04FEF50E00EC0B5
:1005B000A091AE00CA9E412D000C441F50E008F0EF
:1005C00012C04FEF50E00FC05695479594FF07C0FB
:1005D000552309F04FEFA42FA6954A0F521D4F3F08
:1005E000520508F04FEF40939700816061FF09C00A
:1005F000AFE1A095A923AB299A2F8F7DBB2009F4E9
:100600008062A8E1A093680085FF03C0AAE0A093E0
:10061000680061FD03C085FD01C08F7E85FD03C0BC
:10062000A6E0A0936900F894A9B7A160A9BF84FFD0
:1006300002C0A0E4ABBF3FBE189511E00AC013E0B2
:1006400008C01AE006C01EE104C014E602C018EC9F
:1006500000C005E1BB27BA95F1F70A95D9F71A95BD
:10066000C1F708952AE338E709C020E33CE806C053
:100670002AE234EB03C025E238EC00C012E095FD1D
:100680009F7D95FF9062BB27AD9ABA95F1F7AC9A22
:10069000BA95F1F7AC98BA95F1F7AD98BA95F1F72C
:1006A000959AB091AF00BA95F1F79598B7E8BA95D9
:1006B000F1F71A9521F7022FB22FBA95F1F70A95A3
:1006C000D9F73A95D9F6AD9A0895221B39E0001F63
:1006D0003A9509F40895221F211B18F4210F8894DC
:1006E000F6CF0894F4CF622C722CB0E08894B395C6
:1006F000221F331FE0F7379527958894912E802E7F
:10070000020B130B10F4192D082D10F4889401C05E
:100710000894661C771CBA9571F7172D062D08955D
:10072000322D11232AF43A9500951095031B130BD3
:10073000F894029F712C002D129F912C802C78949C
:10074000780C172D921C292DB4E06B2E2695179549
:1007500007956A94D9F7332321F000951095031B70
:10076000130B08950091B6000430A1F1B0919700E9
:10077000B15008F010C0B0916100B09363002092B6
:100780007F0020928000209281002092820020929F
:1007900083006F7B1FC06090B6006064B091610001
:1007A000B093620008E317EC20917A0030917B004F
:1007B00036952795B62DBA9541F036952795B62DE5
:1007C000BA95BA9511F0369527958DDF00937F0085
:1007D00010938000089500917F00B09162000B1B80
:1007E00010918000120928F40038BFEF1B0740F079
:1007F00009C00F37120508F405C00FE710E002C06A
:1008000000E81FEF00938400109385000895009185
:100810008400B09181000B0F10918500B09182008F
:100820001B1F20E03091850033230AF42A95B091F4
:1008300083002B1F1AF4203F40F00AC02F3008F429
:1008400007C00FEF1FEF2FE003C000E010E020EF24
:1008500030916300B0919C003B1718F4323030F0B7
:1008600009C0B0918500BB235AF004C0B091850047
:10087000BB2332F400938100109382002093830005
:1008800008952091D80000918400000F10918500F8
:10089000111F46DF11232AF40038BFEF1B0740F079
:1008A00009C00F37120508F405C00FE710E002C0B9
:1008B00000E81FEF002352F0B0916200B01B0B2F35
:1008C00018F0013008F00AC001E008C000950F5F81
:1008D000B09162000B0F08F001C00FEF009386008B
:1008E00008952091D900009182001091830018DFB3
:1008F00011232AF40130BFEF1B0740F009C00F3F5E
:10090000120508F405C00FEF10E002C001E01FEF70
:10091000112352F0B0918600B01B0B2F18F001305C
:1009200008F00AC001E008C000950F5FB091860092
:100930000B0F08F001C00FEF0093630008950FEF55
:10094000677F71FD29C072FD09C06860B0917B00AE
:10095000BA3020F0B52DB03408F4677FB091D500DF
:10096000BB23D1F0B0917B00BB23B1F00FEF10910E
:100970007B00ABDEF894B091730072FDB5E00B9F85
:10098000112D002D7894112309F00FEFB0919F00E5
:100990000B1710F400919F0000939E0008950091A2
:1009A0007A0010917B0000541140B0919E0010F429
:1009B000BA9501C0B39511F0B0939E00089500C0A0
:1009C00008952091B700B6B1B6FDFBCF04B115B1C3
:1009D000B6B1BF77B6B9B091AC00B395B093AC00E7
:1009E000B83060F12092AC00B091D400BB2321F16B
:1009F000112329F0B091AD00BF3F61F009C0B09163
:100A0000AD000B1739F020F4BB2321F0BA9502C0DA
:100A1000B395E1F300919C00B093AD00BA3750F468
:100A200000ECBF3638F400E8B43620F400E4B93501
:100A300008F400E000939C00777F089510919C00DB
:100A4000B0E11B0F08F41FEF10939C00B091B600AB
:100A5000B43081F000919C00B0916300B01B10F4A1
:100A600000916300B0919E000B1708F00B2F502EE1
:100A700000936400B091AC00B73009F47860089539
:100A800002E3F894B091DA000B9F012D000C001FD7
:100A90007894B0919C000B1710F000919C0000938B
:100AA000610000936300502E0093640000939F0048
:100AB000089520927A00B0EFB0937B000895F894E7
:100AC0000CB51DB52091740078943091750060903C
:100AD00076000093750010937600031B160971FDD4
:100AE00003C076FD81C02BC0709077002093770003
:100AF0002709222311F00FEF1FEF809078009090CC
:100B00007900309378006092790069181619109373
:100B10007C00009175001091760008191909209148
:100B20007A0030917B0036952795020F131F10F441
:100B30000FEF1FEF00937A0010937B0029C02091E4
:100B40007A0030917B003901B4E08B2EB2E09B2E0D
:100B5000343010F08A949A94383010F08A949A9431
:100B6000769467948A94E1F726193709992021F041
:100B7000169507959A94E1F7200F311F20937A007C
:100B800030937B0028F43FEF30937A0030937B0062
:100B9000323008F4706471FF02C0B3E00DC0B09150
:100BA000C60000917100023838F0B395003A08F0A1
:100BB000B395B63008F0B5E09B2EB4E08B2E1091C3
:100BC0007B0000917A0024E0169507952A95E1F7BD
:100BD0000819120928F0B02FB250B12FB20910F441
:100BE00002E010E0980126C020917A0030917B004D
:100BF000390176946794669466946694261932094E
:100C000006950695200F321D20937A0030937B00C5
:100C1000323008F07F7B04E036952795369527958E
:100C200026952695201B10F0223008F422E0890139
:100C30009090C60060FDFECFE0908C00F0908D009B
:100C40006160B9B7B061B9BF380176FD44C0769430
:100C5000679400938C0010938D00B92DB330E1F0B0
:100C6000B0FD04C0060D171D930106C0000F111F33
:100C70000250120922E030E0B92DB33068F0209321
:100C80008E0030938F00009388001093890060924B
:100C90008A0070928B003DC000938E0010938F00ED
:100CA000209388003093890060928A0070928B00B4
:100CB00071FF10C0B0916D00B33060F000918F00F3
:100CC00010917C001595010F28F022F020928E00E3
:100CD00000938F001EC0669400938C00B92DB33032
:100CE00091F0B0FD03C0060D262D03C0000F025089
:100CF00022E0B92DB33038F020938E0000938800A5
:100D000060928A0006C000938E0020938800609253
:100D10008A0000917D0002FD0350013029F495FD09
:100D20000AC0B6E0B7B909C0023019F4B7E0B7B9E4
:100D300004C095FDF6CFB0E0B7B90091A400000F54
:100D400010F4BBE60B270093A40060FDFECFB2E0D9
:100D5000B0936E006160B9B7B061B9BFB72FB6701C
:100D6000A1F020917A0030917B0036952795F89478
:100D70000CB51DB5020F131F1BBD0ABD6160B0E1AC
:100D8000B8BFB9B7B061B9BF7894089560612092D7
:100D90007E0020E067FD20E206C0606120927E00B8
:100DA00020E267FD20E0789401E076FD11C0B72FC6
:100DB000B67009F06F7EB0917B00B55048F002E04C
:100DC000B55020F003E0B55008F006E071FD0AE0F0
:100DD00060FD12C0B0917E00BB2371F071FF08C0AE
:100DE000B0916D00B33020F0B0916E00BA9519F457
:100DF000789470615CC0AEDF789400000000F894D5
:100E000076FD16C010917B00173008F017E0B5E0B2
:100E10001B0F72FD10E183FF110F62FF110F71FDB7
:100E200012E8B4B56090A100B61990F2B10B80F24F
:100E3000B0B7B77FB0BFB8B1B0B7B860B0BFB0910E
:100E40007E00B395B0937E00B8B176FD06C0B1E0E8
:100E500071FDB2E0BA95F1F7B8B1B072B21709F00E
:100E60001BC071FF05C003950A3008F00395B0CF91
:100E700064FF99CF6F7E3CB56DB470907A0080901E
:100E80007B00370D681C6BBC3ABD6160B0E1B8BF38
:100E9000B9B7B061B9BF87CFB0916D00B23008F477
:100EA00082CF64FD80CF0A9509F092CF7F7E20919A
:100EB0008E0030918F00F894B0E1B8BF0CB51DB52D
:100EC000020F131F1BBD0ABDE0908800F09089003F
:100ED0006160B9B7B061B9BF7894B72FB67039F017
:100EE000B0916D0072FFB395B0936D0009C074FFAF
:100EF00007C067FD05C064FD03C0BF91BF91DDC49D
:100F0000089500E063FF03C064FF01C001E0F894AE
:100F100010917100B7E01B9F212D102D7894200FA8
:100F20002695179526951795269517951093710078
:100F3000183718F4B8E7B093710000917100B091C0
:100F400072000B1720F060629598AC98C09860FD15
:100F5000FECFE0908A00F0908B006160B9B7B0617D
:100F6000B9BF0895B2E095FD07C0F894B0937D0035
:100F7000AD9A94987894E5C0F894B0937D00AD9ABA
:100F8000AB987894DEC0B3E082FF24C095FD11C019
:100F900002E0F894B0937D00E7E8F0E00093B3003E
:100FA000C098AB9A62FF02C0AC9A01C0AD98789429
:100FB000C8C002E0F894B0937D00E7E8F0E0009349
:100FC000B3009598949A62FF02C0AC9A01C0AD98A4
:100FD0007894B7C095FD0BC0F894B0937D00E1E71D
:100FE000F0E0C09862FF01C0AC9A7894AAC0F8946F
:100FF000B0937D00E1E7F0E0959862FF01C0AC9A04
:1010000078949FC0B4E095FD07C0F894B0937D003C
:10101000949AAB98789495C0F894B0937D00AB9A6D
:10102000949878948EC0B5E082FF24C095FD11C0DD
:1010300001E0F894B0937D00EDE7F0E00093B30099
:10104000AC98AD9A62FF02C0959A01C094987894CA
:1010500078C004E0F894B0937D00E1E9F0E00093FB
:10106000B300AC98AD9A62FF02C0C09A01C0AB98C1
:10107000789467C095FD0BC0F894B0937D00EBE6C3
:10108000F0E0AC9862FF01C0959A78945AC0F89449
:10109000B0937D00E7E7F0E0AC9862FF01C0C09A32
:1010A00078944FC0B6E095FD07C0F894B0937D00EA
:1010B000AB9AAD98789445C0F894B0937D00949A1B
:1010C000AD9878943EC0B1E082FF24C095FD11C078
:1010D00004E0F894B0937D00E1E9F0E00093B30000
:1010E0009598949A62FF02C0C09A01C0AB98789418
:1010F00028C001E0F894B0937D00EDE7F0E00093A4
:10110000B300C098AB9A62FF02C0959A01C0949850
:10111000789417C095FD0BC0F894B0937D00E7E775
:10112000F0E0959862FF01C0C09A78940AC0F894E4
:10113000B0937D00EBE6F0E0C09862FF01C0959AA5
:1011400078946F7D08952AE630E0F9012092B3008B
:101150009598AC98C098949AAD9AAB9A6B7F089585
:10116000A4EBB0E009E00D9309E00D9304E00D93CA
:101170000FEF0D9303E00D930FEF0D9309E00D9327
:1011800003E00D9301E00D9301E00D93A0ECB0E0BE
:1011900001E00D930FEF0D930D930D930D930D93B0
:1011A00003E00D930FEF0D930FEF0D930D9305E2F9
:1011B0000D9300ED0D9308E20D9300E50D9304E00F
:1011C0000D930FEF0D9302E00D9300E00D930AE7EE
:1011D0000D930FEF0D9300E00D9301E00D9300E0F0
:1011E0000D9303E00D9308952091BB008B7F233076
:1011F00009F48460B091BC00B33019F09F7DB1FD5B
:1012000090629F7BB091BD00B1FD9064223011F0DF
:10121000886001C0877F08950A95E00FF21DB491A0
:101220000895ECE1F0E00091B400F6DFB093D8004F
:10123000ECE1F0E00091B500EFDFB093D900EAE215
:10124000F0E00091BA00E8DFB093DA00B091D0008E
:101250000FEF1CE0B23011F400EA1AE0B33011F4E1
:1012600002E815E00093720010937300E8E3F0E0E9
:101270000091D700D1DFB093A20008950895209186
:10128000CA003091CB00B091BC00B33009F43E509D
:1012900097FF02C020E03FEFB32FB21B6B2EB25876
:1012A00010F4B2E86B2E00E00395609EB12DBD579F
:1012B000D8F30093AE0008959068E1DFC4D920E030
:1012C00030E0B0E16B2EBBD9B09197002B0F321DEF
:1012D0006A94C9F7B4E036952795BA95E1F7822E5E
:1012E0009F77CDDF0895F894E3E0F0E0B9E0B7BF71
:1012F000B491B078C1F3F894A895B1B5B861B1BD17
:10130000B0E0B1BDB4E0BEBFBFE5BDBF1CDFB0E023
:10131000B8BBB1E1B7BBB8E2B5BBB8E3B4BBB0E1B1
:10132000B2BBB0E3B1BB2224A0E0B0E02D92AA3161
:10133000E9F7A0E6B0E00FEF2D920A95E9F7B1E0EA
:10134000B093A4000DDFE9D2B6B1B460B6B9009194
:10135000CC000093AF00B1E0B0936A00F89477D965
:1013600081D971D982D96FD983D96DD9F8940AEF0F
:101370001AEFA0B396FDA095A2FF1FC01A95C9F75A
:101380000A95B1F7E0E0FCE1B591B43E39F4B591CE
:10139000B03E21F4B591BF3F09F40CC0E0E0F395F5
:1013A000F395B591B83F49F4B591B43931F4B5919D
:1013B000BA3A19F4EE27F695099416DF32DF5EDFAC
:1013C0005EDF0091CC000093AF00BDDEB2E0B3BFA2
:1013D000B2E0BEBDB2E0B5BDB1E5B8BFB9BFB0B710
:1013E000B77FB0BFB8B1B0B7B860B0BF26D97894F6
:1013F000E6DAB3E096FDB2E0B5BFB0E4BBBFBB2711
:10140000B064BABF8D7F23D9626033E02CE0B09125
:101410009600BB2321F42CE03A9509F4A7CF13D909
:1014200080FFA4CF8E7FB0919700B23078F3B92FB0
:10143000BF710091990000939800B0939900B01784
:1014400029F72A9521F76D7FB3E096FDB2E0B5BF8D
:10145000BB27B064BABF8D7FB091D600BB2321F407
:101460008062B92FB0709B2F8F7B20926700EDD8E0
:1014700085FF05C0B0916700BA3008F08064DFD8FE
:1014800002E085FF01C000E0B0919700B017B8F30B
:10149000F894E8D8E7D8E6D87894D9D8209287008D
:1014A000B091BC00B33009F474C0C9D8B091C00089
:1014B000B13008F46EC0B0916A00B13008F469C070
:1014C00085FD18C0B0919700BF3F08F462C0F89442
:1014D000D2D87894BAD8B0919700B130C0F7F894C8
:1014E000C1D8AFD8BFD87894B0D8B0919700BF3FDB
:1014F000B0F3D4C2B3E09B2E9068F894C0DE789429
:10150000A4D8F8949F77BBDE80909700B0919700A5
:10151000BF37789408F445C090D8F894ACD8789444
:101520009A9451F7C9DEB82DB550B093CB008FD83F
:10153000F89420D286D27894BAE09B2E9068F894E2
:101540009EDE789482D8F8949F7799DE80909700F9
:10155000B0919700BF37789478F76FD8F89482D815
:1015600070D880D878949A9449F7A6DEB82DBB5FDE
:10157000B093CA006CD8F894FDD172D2789465D833
:10158000F8947DDE7894B0919700BF3F08F498CF2F
:1015900085C200919700B09187000B1710F000935F
:1015A000870053D801E0B091BC00B35009F405E0C6
:1015B000B0919700B01708F073CFF8945CD85BD85F
:1015C0005AD8789444D820926A0020926B002092D6
:1015D0006C00B0916B00B395B0936B00BF3F69F5A1
:1015E000B0916C00B395B0936C00B091CE0009E15E
:1015F000BA9559F002E3BA9541F00DE7BA9529F092
:101600000AEFBA9511F020926C00B0916C00B017FF
:10161000A0F0B0916C00BA95B0936C00B4EBB093AD
:101620006B00B091CD00B093AF00F89424D87894BB
:10163000B091CC00B093AF0008D803D8B091680047
:10164000BB2319F485FF01C091CE01E085FD01C0E7
:1016500006E0B0919700B01708F4BBCFB091BC0082
:10166000B35009F0F2D7B0916800BB2309F47ECEE5
:10167000F89469DD2092610020926200209263005C
:10168000522C209264002092A3007894B091B9006B
:10169000BB0FB093A00020927F0020928000209288
:1016A000810020928200209283002092AC0060E0B2
:1016B00070E020927100B8E0B093AC007860BDD7C4
:1016C000B2E073FDB1E0B7B9B6B1B068B064B6B915
:1016D000B6B1B6FDFDCF04B115B1B6B1BF77B6B99D
:1016E000112309F00FEF0093AD006BD9B8E0B09370
:1016F000AC0078608090BB00B2E0B093BB0074DDBA
:101700008092BB00F894BFEFB0939C00B9D9B09120
:101710006100B0939C00B0939D00B0939E007894BC
:10172000B1E0B0936100B09363005B2EB0936400AE
:10173000B093A600B0919B00B093A500B091BC00FF
:10174000B33019F49F7D87FD9062716072602092C2
:101750006D00A8DCB8DCADD9B2D9ABD9B0D9A9D964
:1017600006C0F89441DD78942092AC00777F15DBB9
:10177000F9D7C7DBF7DBA3D909DB66FD2CD876FFE9
:10178000DED876FD0CD9BDDBFEDB99D906DB66FD24
:101790003ED8B7DB37DC93D9F9DA66FD72D8B1DB16
:1017A00042DC8DD9FADA66FD9CD8ABDB7BDC87D9CD
:1017B000EDDAB2E073FDB1E0B7B9B6B1B068B064CC
:1017C000B6B99FDB80DC7BD9FCD871FF26C067FDF2
:1017D00024C0B0919F00B0939C00B0939D00B09145
:1017E0009B00B093A500B1E0B093A60018E12CE0F7
:1017F000B0916D00B11758F07D7F746020936F0039
:10180000B0919F00B0939C00B0939E0006C0B09131
:101810009700B13008F0ABCF5AC072FF10C067FD1F
:101820000EC0B0916F00BA9511F47B7F9ACFB09340
:101830006F00B0919700B13008F099CF48C0209266
:101840007000B0919A000AEFB01708F040C085FF11
:1018500004C0B0916800BB23D1F1B091BC00B3309B
:1018600081F495FD03C087FD04C00BC087FF01C054
:1018700008C067FD06C06068B0919F00B0939C00EF
:101880008BCF00EF67FF05C0B0919F00B0939C0025
:1018900000E2B0917B00B01708F469CF67FF17C072
:1018A0006F779F7D87FD90627460B2E1B0936F00A7
:1018B000B0919F00B0939C005ACFB0917000B39547
:1018C000B0937000B0919700BB2309F002C0209242
:1018D0007000F89438DC8090BB00B2E0B093BB009D
:1018E00083DC8092BB0020926100209262002092F3
:1018F0006300522C209264002092A0007E7F789496
:101900009CD621DCB6B1B460B6B985FF05C0B091F4
:101910007000B53008F02ACD58CEEDE0F0E023D0CD
:10192000053509F01BC0EEE0F0E01DD00A3A09F0E1
:1019300015C03AE0A4EBB0E0E3E0F0E014D00D9382
:1019400031963A95D9F738E1A0ECB0E0EFE0F0E05D
:101950000AD00D9331963A95D9F702C001DC0AD02E
:10196000E7E2F0E00895E199FECFEEBBFFBBE09A1D
:101970000DB308951ED03AE0A4EBB0E0E3E0F0E050
:101980000D910FD031963A95D9F738E1A0ECB0E03F
:10199000EFE0F0E00D9105D031963A95D9F712D0ED
:1019A0000895E199FECF0DBBEEBBFFBBE29AE19A31
:1019B0000895EDE0F0E00FEFF4DFEEE0F0E00FEF80
:1019C000F0DF0895EDE0F0E005E5EBDFEEE0F0E0BC
:1019D0000AEAE7DF08953091B0000091B10031309C
:1019E00011F40093B400323011F40093B500333099
:1019F00011F40093B600343011F40093B800353080
:101A000011F40093BA00363011F40093C600373059
:101A100011F40093BB00383011F40093D700393033
:101A200011F40093D0003A3011F40093BC003B3025
:101A300011F40093BD00089525E009D62A95E9F731
:101A4000089510D612D614D616D6FBD50BD60DD6C1
:101A50000FD611D6F6D506D608D60AD60CD60895D6
:101A60000AD606D602D6FED5ECD505D601D6FDD5CA
:101A7000F9D5E7D500D6FCD5F8D5F4D508958090F2
:101A8000B0009090B100EED5EDD5ECD5DAD58A94C2
:101A9000D1F7F1D5D6D59A94E1F70895F894D1DF2E
:101AA0007894CADFC9DFB1E0B093B000B1E0B09381
:101AB000B1002092B200F894E2DF7894B5E06B2E8A
:101AC00070909700C4D5B09197007B16C9F7B130DC
:101AD00018F0BF3F40F107C07EDFF8944BDFB1DF65
:101AE000B8E0B1BDA9DF6A9459F7B091B200B395DF
:101AF000B093B200B33008F4DECF9EDFB091B100F6
:101B0000B395B093B100F894B091B000BA95EEE3FC
:101B1000F0E0EB0FF21D049178940395B091B100C1
:101B2000B01708F4C6CF88DF87DFB091B000B39557
:101B3000B093B000B091B000BC3008F4B7CF10DB68
:0C1B4000F89418DFB8E0B1BD77DFCDCB22
:00000001FF
